:020000020000FC
:1000000003C0C0C118954FC110E0B59B106890E8BF
:1000100098B993E093BF90E09EBBE09A2DB3287708
:100020003327442755276627772788279FEFA92E50
:100030000FEFAA2790E092BF92E099BF9FEF492E61
:1000400090E097BB2877FF27EEE3E199FECFEEBB68
:10005000E09A9DB3F90FEA95EF3FC9F79FE39EBB86
:10006000E09A9DB3F91709F41160E1E010FF03C0B5
:1000700024FD01C08DC01EC0FF27EEE3E199FECF35
:10008000EEBBE09A9DB3F90FEA95EF3FC9F7E1990E
:10009000FECFEFE3EEBBFDBBF894E29AE19A7894D1
:1000A000116008C0912F9073E90FEEBBE09ABDB3C9
:1000B000B3D000C027FDD4C021FF03C02D7FE2E0F4
:1000C00067C0B29909C022FD08C0246010FF05C0B6
:1000D00026FD03C0E3E05CC02B7F92E295BF90E475
:1000E0009BBF7894889520FFE5CF2E7FB9C090F50F
:1000F000EB2FEF70F0E0B07FB03111F1B03221F1B1
:10010000B03351F1B034C1F1B03561F2B03611F411
:10011000E22D41C0B03739F490E09EBBE09A9DB328
:10012000907F292BA9CFB03831F4B0E0889474D0F7
:10013000B1E172D0BFCFB03911F4BD98BBCFBACF07
:1001400092E0E90F2082B6CF92E0E90FB081889467
:1001500063D0B0CF2B2EAECFF12F1260B52D5CD077
:10016000B62D5AD0B72D58D0B82D56D0B92D54D061
:10017000BA2D52D01F2F9ECFE199FECF912F9073B1
:10018000E90FEEBB2DBAF894E29AE19A789492CFF7
:10019000EEBBE09AEDB317FD24C0EEBBE09A9DB331
:1001A000913001F1923009F4BD98933009F4BD9A71
:1001B000943029F4E395EEBBE09A9DB3192B95306A
:1001C00029F4E395EEBBE09A9DB319239C30B9F076
:1001D0009D3011F4339403C09F3F19F0D6C0E395CE
:1001E000DACF68CFF12F1260AA24992488247724CB
:1001F00066245524146012FDFECF1F2FF0CFDBE0E4
:10020000E395EEBBE09A9DB3CE2FED2F9083EC2FBC
:10021000D395D131A9F7E3CFD9E092E0092E277F1A
:1002200023FD1DC0B19BFCCFB89810F0C098B89AC0
:1002300023FD15C0C198B99A2FD0B9982DD0B19986
:10024000F7CF10F0B89802C0C098B89A23FD07C045
:10025000B19BFCCFB898BB1FDA9511F70895F0CE8B
:10026000D9E092E0092E277F23FD1AC0B199FCCF77
:10027000C198B99A8894B09B06C0089423FD10C019
:10028000B099FCCF04C023FD0BC0B09BFCCFB99844
:10029000BB1FDA9549F72BCFC1E0CA95F1F7089556
:1002A000B9982F7707CF1FB6AA2311F4A1E067C032
:1002B000002021F00A9411F428602F7712FF07C064
:1002C0003A2D492D582D672D762D852D1B7F13FD39
:1002D00055C033953C3309F027C0332743954C3341
:1002E00009F022C044275395583109F01DC0552705
:1002F0006395603299F06F3141F4743079F0763063
:1003000069F0793059F07B3049F0723069F46E3120
:1003100029F06D3149F4A82FA37031F061E0739595
:100320007D3011F471E0839511FD06C0A32E942E4B
:10033000852E762E672E582E16FF20C0A42DA79549
:1003400010F43017D9F4A79510F44F15B9F4A79508
:1003500010F45E1599F4A79510F46D1579F4A7952E
:1003600010F47C1559F4A79510F48B1539F410FF8F
:1003700004C025FD02C0226001C0BD9AAA272E7FBD
:100380001FBE18952160206818959E3021F4E395D2
:10039000EEBBE09A4DB29F3021F4E395EEBBE09ABC
:1003A0003DB2903109F43A9497FF25C0E395EEBB36
:1003B000E09ABDB396FF04C0E395EEBBE09ADDB3CF
:1003C000903C11F43D16C1F0913C11F43D16A1F49E
:1003D000903809F411C0913811F4321469F0923850
:1003E00011F4321449F4933811F4B2992AF4943880
:0C03F00011F4B29B0AF4F3CEEB2FCDCE3B
:00000001FF
